:020000040000FA
:06000000FE300F306A28FB
:08000800A000030EA100831209
:10001000C31D3B288B1C34288B1031181628B11CAB
:10002000342864300102031833281A2800001828E5
:1000300019281A281B281C281D281E281F2820289C
:1000400021283110B114A810031005190314AA0DAA
:10005000A90DA80DB00B342831152A08AF002908C6
:10006000AE002808AD00B11081010B11210E8300F4
:10007000A00E200E090005194328831601178312CC
:10008000B23081005E2883160113831203140B190A
:100090000310A80DA90DAA0DAB0DAC0DAC16FF30C9
:1000A0002C02031D5E28FA302B02031D5E28311539
:1000B0002A08AF002908AE002808AD008B100B11EC
:0A00C000210E8300A00E200E09009F
:0C00D400203084008001840A8030040287
:1000E000031C6C281230B0005A30C000C10001302F
:1000F000D400D500E400E500E300F100F000073093
:10010000D8008030D7001F30E6000717FA30FD0016
:100110000330EF0083160F308505203086050D3043
:1001200087058312850186018701103083168E00B2
:100130008312703083168F008312003003179900EA
:100140000313003003179A000313003097000030A8
:100150009F00003083169F008312003003179E001B
:100160000313003003179F000313C0308316810070
:1001700083123130900000309200003083169400DA
:10018000831200309400A63083169800831200304A
:1001900083169B00831290309800333083169900A9
:1001A0008312003083168C008312003083168D007A
:1001B000831210308B000D16252581018E018F01D1
:1001C0000B118B100B108C128C018D010D168B17DF
:1001D000052343237A2125213119B823311A3F21E0
:1001E000591CE822591879228F080319EB288F012E
:1001F0003E18A324BB227923F621D1219121B121DC
:100200000829E71BEB01EB0B0829E801E901EA01EA
:10021000E7135918EB28B1191A29D60BEB28B11A94
:100220000A30B11EC830D600B11A21297A21CC0A71
:10023000CC194A14B111B11A0A30B11EC830D60017
:10024000EB287A21BE182525EB286400C31DB113C5
:10025000C31D0800311808000B1D08000B11B11058
:1002600031141230B000051D3A29B117831601135D
:1002700083120800B113831601178312080031128C
:100280004A10CC0121305B02031D4C295C08CE00D2
:100290005D08CF00661775295B085C065D02031DCB
:1002A000080077305B02031D59295C087406C400FE
:1002B000752966305B02031D60295C08CB00752937
:1002C00055305B02031D67295C08F800752944302E
:1002D0005B02031D6E295C08FA00752933305B024E
:1002E000031D75295C08FB007529B116B1110A3090
:1002F000D6000800591459158B1383160712831260
:100300008B17071608005910D9101930DE00B112EA
:10031000B111C830D6008B138316071683128B17C2
:100320000800051898291930C00703189D290800EE
:100330000A30C002031CA9290800FF30C000421483
:1003400064304102031808004210C2144317C3145A
:100350000800C0014210C213C21C0800C2014313AE
:1003600008008518B8291930C1070318BD290800ED
:100370000A30C102031CC9290800FF30C100421421
:100380006430400203180800421042154317C3109E
:100390000800C1014210C213421D0800C2014313EC
:1003A0000800E303031D080065186008E5186108EC
:1003B0006519620899000330E3000310E50DE519A3
:1003C000E22908001430E3000130E5001030E61A9D
:1003D000E4002030661BE4000310E40D03186414ED
:1003E000640866050319E229052308008C1E08002D
:1003F000E7174A150717FA30FD001819CA146908DB
:10040000E8006A08E9001A08EA00E81F080068081E
:10041000C13C031D122A69086A05C3046A096904FC
:10042000C305782A6808C23C031D1D2A69086A05AD
:10043000C5046A096904C505782A6808C43C031D17
:10044000242A6908F700782A6808FC39E03C031D73
:10045000342A690868188038BB006A08E8188038B0
:10046000BA000925BE14782A6808FC39F03C031D3F
:100470004E2A690868188038EC0064000D1E3E2A78
:100480008B136C0803178D0083168C130C148312C6
:100490000C080313ED008B17E616782A6808FC3960
:1004A000803C031D5D2A690868188038CE006A0800
:1004B000E8188038CF00D815782A6808FC39903CB5
:1004C000031D682A690868188038CE005816782AF3
:1004D0006808A03C031D782A69086A188038CD0096
:1004E000C310EA18C31445126A194516D816782A9B
:1004F00008005919862AD3030F305305031D08003D
:10050000D3080319892A0716D30E0800591B4F2355
:10051000591307125911D918832955185008D5189D
:100520005108551952085705031D992AFF30D30069
:100530009C2A2230D3009C2A0310D70C0318A12A2E
:1005400008008030D7000310D50DD519A82A08005F
:100550000130D5000430D819D4000830581AD4001E
:100560000310D40D03185414540858050319A82A6D
:100570004323D9140800EF0B08000330EF00061ED8
:10058000E62A05160310F00D031CD42A0130F000F2
:100590000310F10D711ED42A0130F100F00044085F
:1005A000F300C31AF317051271187308F1187208D3
:1005B00071197708F11DDF2A4B084A188038700539
:1005C000061203198516031D851208000616080079
:1005D000DA0A0319D9165916071E5912D91D012B0B
:1005E000591A012BB1155A08283CD91A0310DD0DF0
:1005F000DC0DDB0DDA01D912DE0B012B31161930BF
:10060000DE00D915591ED9110800E001E101E2010F
:10061000641F112B4830E0004E08E1004F08E20053
:100620006613E41E1A2B4730E0006C08E1006D08E9
:10063000E200E612641E222B4130E0007A08E1005D
:100640007B08E200E41D2A2B4C30E0007708E10033
:100650007808E200641D322B4530E0004A08E100D2
:100660004B08E200E41C3A2B4630E0004308E1006E
:100670004408E200641C422B5830E0005930E1008D
:100680005A30E2000800D001D101D201541C4D2B98
:10069000F730D0004308D100752BD41C542BA13067
:1006A000D0007708D100752B541D5B2BA230D000F1
:1006B0004508D100752BD41D652BC130D0004E08E4
:1006C000D1004F08D200D8110800541E6D2BC23043
:1006D000D0004E08D1005812752BD41E0800A73048
:1006E000D0004D08D100D812752B50085106D20009
:1006F0000800311F7E2BFC0303193113071F832BC6
:10070000FD0303190713031044180314B20DF0304E
:1007100032020319431307184311071C4315071925
:10072000C311071DC315751C992BC31E8710C31A4F
:100730008714FE0B080044187325441C87124A1CBA
:1007400087174A186B25790AF71BF707771BAC2B1D
:10075000790A77020318F7007808F2000310790C81
:10076000013E7802C3120318F2000318C3160800F2
:100770003111311B0800591808004A100717FA30C8
:10078000FD00B7010430B8000C30370230300318D8
:10079000B807C319B8178B1320303707380703176A
:1007A0008D0083168C130C1483120C080313A40001
:1007B000A500C030A50610303707380703178D0095
:1007C00083168C130C1483120C080313A300A600C9
:1007D0000230A60600303707380703178D0083164E
:1007E0008C130C1483120C080313A200A700013011
:1007F000A7068B17B11F022C22090339A200A309F7
:10080000A409A509C31D112C22082D02031D9D2C2E
:1008100023082E02031D9D2C24082F02031D612C8A
:100820001D2C24082F02031D9D2C23082E02031DBE
:10083000612C22082D02031D9D2C00303702031D60
:10084000272C3D18272C3D143E144314080001307A
:100850003702031D352CFF30FC003117431FC31432
:10086000431FEC244030C306080002303702031D4A
:10087000432CFF30FC003117431FC314431FF424E3
:100880004030C306080003303702031D4A2C431FC3
:10089000C314080064000D1E4B2C30303707380796
:1008A0007F3903178D0083168C130C1483120C08E8
:1008B0000313F7005917AA24FF30FC00311740300A
:1008C000C306C31D682C25082F02031D9D2C702C08
:1008D00026082E02031D9D2C27082D02031D9D2C8A
:1008E00000303702031D7A2C3D1C7A2C3D103E143B
:1008F0004310080001303702031D882CFF30FC0034
:100900003117431FC310431FE3244030C3060800C0
:1009100002303702031D962CFF30FC003117431FB5
:10092000C310431FF4244030C306080003303702CD
:10093000031D9D2C431FC3100800B70A1C3037024B
:1009400003180800C22B3E102330BB004508BA0034
:1009500009250800771B0800871D08000310790C83
:10096000013E77020318F7000318AE2C77087802CF
:100970000319CC2C0318C42C78087702C318790209
:10098000C318013EFF00D22C77087802C31C7902FD
:10099000C31C013EFF00D22C0310790C013EFF0066
:1009A000F70708000310790C023E7F02031C0800C1
:1009B0000310790C013EF707790A77020318F70054
:1009C0000318DC2C08005917C310780AF700790ABD
:1009D00077020318F70008005917C3147803F700CB
:1009E000790AF71BF707080059170310790C7807E5
:1009F0007902031C032D0319032D0310790C013E0A
:100A00007807F70008000310790C013E7802F70020
:100A100008000D123B08831203178D008312031385
:100A20003A08831203178C00831603178C130C15D6
:100A30008B138B1B182D55308D00AA308D008C1414
:100A40008B170C1183120313080064000D1E262D52
:100A5000BE108B138B1B292D313003178D0083168D
:100A60008C130C1483120C080313F4008B177410EE
:100A70008B13323003178D0083168C130C148312E2
:100A80000C080313F5008B178B13333003178D00FD
:100A900083168C130C1483120C080313F6008B17A7
:100AA0008B13233003178D0083168C130C148312C1
:100AB0000C080313C5008B178B13303003178D0000
:100AC00083168C130C1483120C0803130718303090
:100AD000F900F90308000708803A870008000708B2
:100AE000403A870008000708203A870008000708F6
:060AF000023A8700080035
:084000000F00000002000700A0
:02400E00CC03E1
:1042000000002700FF00FF0040004200440046007D
:104210004200430040004100460047004400450082
:10422000FF00FF00FF00FF00F200F600FA00FE00B2
:10423000F000F200F400F600F800FA00FC00FE00C6
:10424000FF00FF00FF000000E500E500E500E500DD
:10425000E900E900E900E900E900E900E900E90016
:104260001800000001000000FF00FF00FF00FF0039
:104270000000010002000300040005000600070022
:104280004300420041004000470046004500440012
:104290004400450046004700400041004200430002
:1042A000F000F200F400F600F800FA00FC00FE0056
:1042B000F000F200F400F600F800FA00FC00FE0046
:1042C000ED00ED00ED00ED00ED00ED00ED00ED0086
:1042D000F100F100F100F100F100F100F100F10056
:1042E000080009000A000B000C000D000E000F0072
:1042F0001000110012001300140015001600170022
:10430000FF00FF00FF00FF000000000000000000B1
:104310000300030003000300030003000300030085
:10432000FF00FF00FF00FF00C800C800C800C80071
:10433000C800C800C800C800C800C800C800C8003D
:10434000FF00FF00FF00FF00C300F300CF00FF00ED
:104350000300C3003300F3000F00CF003F00FF0055
:10436000FF00FF00FF00FF00FF00FF00FF00FF0055
:10437000FF00FF00FF00FF00FF00FF00FF00FF0045
:10438000020002000200020002000200020002001D
:10439000000000000000000000000000000000001D
:1043A000C800C800C800C800C800C800C800C800CD
:1043B00088008800880088008800880088008800BD
:1043C0000300C3003300F3000F00CF003F00FF00E5
:1043D0000300C3003300F3000F00CF003F00FF00D5
:1043E000FF00FF00FF00FF00FF00FF00FF00FF00D5
:1043F000FF00FF00FF00FF00FF00FF00FF00FF00C5
:00000001FF
